:0200000480007A
:100000006F008004732F2034930F80006308FF0378
:10001000930F90006304FF03930FB0006300FF038E
:10002000130F000063040F0067000F00732F2034CC
:1000300063540F006F00400093E19153171F0000BD
:1000400023223FFC6FF09FFF93000000130100008C
:10005000930100001302000093020000130300004C
:100060009303000013040000930400001305000034
:10007000930500001306000093060000130700001C
:100080009307000013080000930800001309000004
:1000900093090000130A0000930A0000130B0000EC
:1000A000930B0000130C0000930C0000130D0000D4
:1000B000930D0000130E0000930E0000130F0000BC
:1000C000930F0000732540F16310050097020000B4
:1000D000938202017390523073500018970200000F
:1000E00093824202739052309B021000939252030B
:1000F0009382F2FF7390023B9302F0017390023AF5
:100100007350403097020000938242017390523046
:10011000735020307350303093010000970200007C
:10012000938282EE73905230130510001315F5017F
:10013000635C05000F00F00F930110009308D005D9
:10014000130500007300000093020000638A0200A0
:1001500073905210B7B200009B82921073902230BD
:100160007350003097020000938242017390123462
:10017000732540F173002030B70000801BD70000CA
:10018000B70300809301200063107732B70000802E
:100190001BD71000B703004093013000631677307F
:1001A000B70000801BD77000B70300019301400027
:1001B000631C772EB70000801BD7E000B703020056
:1001C000930150006312772EB70000809B801000CF
:1001D0001BD7F00193031000930160006316772C86
:1001E0009300F0FF1BD700009303F0FF9301700012
:1001F000631C772A9300F0FF1BD71000B703008021
:100200009B83F3FF930180006310772A9300F0FF34
:100210001BD77000B70300029B83F3FF930190008C
:10022000631477289300F0FF1BD7E000B7030400A6
:100230009B83F3FF9301A000631877269300F0FFE0
:100240001BD7F001930310009301B000631E7724C5
:10025000B72021219B8010121BD70000B72321213A
:100260009B8313129301C00063107724B7202121D0
:100270009B8010121BD71000B79390109B8303092B
:100280009301D00063127722B72021219B801012A6
:100290001BD77000B74342009B8323249301E000E7
:1002A00063147720B72021219B8010121BD7E00018
:1002B000B78300009B8343489301F0006316771EC9
:1002C000B72021219B8010121BD7F001930300005F
:1002D00093010001631A771CB720F1FF9B80503413
:1002E0009390C000938080671BD70000B7533412EF
:1002F0009B8383679301C0026318771AB720F1FFCD
:100300009B8050349390C000938080671BD740003F
:10031000B74323019B8373569301D002631677186A
:10032000B72009009B8050349390C0009380806771
:100330001BD70000B75334929B8383679301E0027D
:1003400063147716B72009009B8050349390C00047
:10035000938080671BD74000B74323099B83735664
:100360009301F00263127714B70000809BD07000F5
:10037000B70300019301100163987012130200008B
:10038000B70000801BD77000130307001302120090
:1003900093022000E31652FEB703000193012001EF
:1003A0006314731013020000B70000801BD7E00035
:1003B0001300000013030700130212009302200031
:1003C000E31452FEB703020093013001631E730C65
:1003D00013020000B70000809B8010001BD7F001C3
:1003E00013000000130000001303070013021200A3
:1003F00093022000E31052FE93031000930140018A
:100400006314730A13020000B70000801BD770004A
:100410001302120093022000E31852FEB7030001FA
:10042000930150016312770813020000B7000080A7
:10043000130000001BD7E0001302120093022000FB
:10044000E31652FEB703020093016001631E7704B6
:1004500013020000B70000809B8010001300000012
:10046000130000001BD7F0011302120093022000BA
:10047000E31252FE9303100093017001631677029A
:100480009B50F0019303000093018001639E700074
:100490009300F0011BD0C001930300009301900171
:1004A00063147000631030020F00F00F63800100CE
:1004B0009391110093E111009308D0051385010079
:1004C000730000000F00F00F930110009308D00597
:1004D0001305000073000000731000C0000000004E
:1004E000000000000000000000000000000000000C
:0C04F00000000000000000000000000000
:1010000000000000000000000000000000000000E0
:1010100000000000000000000000000000000000D0
:1010200000000000000000000000000000000000C0
:1010300000000000000000000000000000000000B0
:081040000000000000000000A8
:040000058000000077
:00000001FF
